:020000040000FA
:1000000001288316FF239000C8308500003081004E
:1000100008309600831285010730990008308B0064
:10002000C83081008319772825188028A42025143A
:10003000290D290D291A013AA91A013AA919013ADB
:10004000A900290D290D291A013AA91A013AA9195D
:10005000013AA9004920A501492029088720240840
:10006000952085000630A000A220A00B342880280F
:10007000C830A10050302407A700210E0F39503896
:10008000281BA70B412820308506A10B3A28851292
:100090000034320D320D321A013AB21A013AB21955
:1000A000013AB200320D320D321A013AB21A013A57
:1000B000B219013AB20032088E200630B118310868
:1000C00031193108B1193108311A3108B11A310822
:1000D000311B3108B11B310831183108A0008620CE
:1000E0002408952085003820A00B6F280034A60135
:1000F000173085000630A0003820A420A00B7C28F3
:10010000A4203820A60AA501850163000108A400E7
:100110000C3003102402031887280034B100043087
:100120000310310203188E28003482071034013482
:1001300011340534153407341034043414340534C0
:1001400015340734A301A6280130A3004630A200CD
:10015000A101A10BA928A20BA828A30BA628003453
:040160000034003433
:0207FE000034C5
:02400E00A43FCD
:00000001FF
